:10000000020FD1E4FFFE12014C600C0FEF70010EE5
:0900100009E970F20A80EF2222D6
:07001B0002422D010000006C
:10002300023D1AE4FF0227A2024250EFC3940940A3
:0E00330005EF940E4003BF2003D38001C322CB
:0E004300023F0374FFF0A37400F0A3742022A8
:100053000242BAE709F608DFFA8046E709F208DF49
:10006300FA803E88828C83E709F0A3DFFA8032E3CB
:1000730009F608DFFA8078E309F208DFFA8070886E
:10008300828C83E309F0A3DFFA806489828A83E0A8
:10009300A3F608DFFA805889828A83E0A3F208DF97
:1000A300FA804C80D280FA80C680D4806980F28046
:1000B30033801080A680EA809A80A880DA80E2806C
:1000C300CA803389828A83ECFAE493A3C8C582C8C1
:1000D300CCC583CCF0A3C8C582C8CCC583CCDFE92B
:1000E300DEE7800D89828A83E493A3F608DFF9ECC7
:1000F300FAA9F0EDFB2289828A83ECFAE0A3C8C552
:1001030082C8CCC583CCF0A3C8C582C8CCC583CC78
:10011300DFEADEE880DB89828A83E493A3F208DFE7
:10012300F980CC88F0EF60010E4E60C388F0ED24B7
:1001330002B4040050B9F582EB2402B4040050AFBA
:1001430023234582239000A673BB010689828A83F9
:10015300E0225002E722BBFE02E32289828A83E483
:100163009322BB010CE58229F582E5833AF583E00E
:10017300225006E92582F8E622BBFE06E92582F82D
:10018300E222E58229F582E5833AF583E49322BBF3
:10019300010FF8E58229F582E5833AF583E028F03B
:1001A300225009C58229F8E58226F622BBFE09C53D
:1001B3008229F8E22582F222F8EA2583F583E9937E
:1001C3002822BB010689828A83F0225002F722BBD0
:1001D300FE01F322F8BB010DE58229F582E5833A9E
:1001E300F583E8F0225006E92582C8F622BBFE0516
:1001F300E92582C8F222EF8DF0A4A8F0CF8CF0A4F9
:1002030028CE8DF0A42EFE22BC000BBE0029EF8D5C
:10021300F084FFADF022E4CCF875F008EF2FFFEE89
:1002230033FEEC33FCEE9DEC984005FCEE9DFE0F97
:10023300D5F0E9E4CEFD22EDF8F5F0EE8420D21CF2
:10024300FEADF075F008EF2FFFED33FD400798503A
:1002530006D5F0F222C398FD0FD5F0EA22C5F0F8D7
:10026300A3E028F0C5F0F8E582158270021583E05B
:1002730038F022BB010A89828A83E0F5F0A3E022E9
:10028300500687F009E71922BBFE07E3F5F009E3FF
:10029300192289828A83E493F5F074019322BB01C6
:1002A3000A89828A83F0E5F0A3F0225006F709A7B2
:1002B300F01922BBFE06F3E5F009F31922F8BB019E
:1002C30011E58229F582E5833AF583E8F0E5F0A3A9
:1002D300F0225009E92582C8F608A6F022BBFE09E0
:1002E300E92582C8F2E5F008F22275F0087582006C
:1002F300EF2FFFEE33FECD33CDCC33CCC58233C5E8
:10030300829BED9AEC99E58298400CF582EE9BFE78
:10031300ED9AFDEC99FC0FD5F0D6E4CEFBE4CDFAD3
:10032300E4CCF9A88222B800C1B90059BA002DEC77
:100333008BF084CFCECDFCE5F0CBF97818EF2FFF0F
:10034300EE33FEED33FDEC33FCEB33FB10D70399B7
:100353004004EB99FB0FD8E5E4F9FA227818EF2F64
:10036300FFEE33FEED33FDEC33FCC933C910D70583
:100373009BE99A4007EC9BFCE99AF90FD8E0E4C9A2
:10038300FAE4CCFB2275F010EF2FFFEE33FEED33D2
:10039300FDCC33CCC833C810D7079BEC9AE89940FF
:1003A3000AED9BFDEC9AFCE899F80FD5F0DAE4CD61
:1003B300FBE4CCFAE4C8F922EB9FF5F0EA9E42F0A5
:1003C300E99D42F0EC6480C864809845F022EB9F7D
:1003D300F5F0EA9E42F0E99D42F0E89C45F022E800
:1003E300600FECC313FCED13FDEE13FEEF13FFD808
:1003F300F122E6FC08E6FD08E6FE08E6FF22E6FB3E
:1004030008E6F908E6FA08E6CBF8227401FF33950B
:10041300E0FEFDFC080808E6CF2FF618E6CE3EF610
:1004230018E6CD3DF618E6CC3CF622ECF608EDF6E0
:1004330008EEF608EFF622ECF0A3EDF0A3EEF0A33E
:10044300EFF022D083D082E493F608740193F60888
:10045300740293F608740393F6740473D083D08202
:10046300F8E4937012740193700DA3A393F87401CD
:1004730093F5828883E4737402936860EFA3A3A364
:1004830080DFD083D082F8E4937012740193700DEF
:10049300A3A393F8740193F5828883E4737402939E
:1004A300B5F0067403936860E9A3A3A3A380D8D02F
:1004B30083D082E4937012740193700DA3A393F815
:1004C300740193F5828883E4737402936C701274DD
:1004D30003936D700C7404936E70067405936F60D0
:1004E300DDA3A3A3A3A3A380CAE3F5F009E208B5A0
:1004F300F06BDFF58067E3F5F009E608B5F05EDF42
:10050300F5805A87F009E608B5F052DFF6804E878A
:10051300F009E208B5F046DFF6804288828C8387D3
:10052300F009E0A3B5F036DFF6803288828C83874A
:10053300F009E493A3B5F025DFF5802188828C834D
:10054300E3F5F009E0A3B5F014DFF5801088828CA1
:1005530083E3F5F009E493A3B5F002DFF402061B8D
:10056300808780E9809080D4803E8015806E807E75
:10057300809D80B7808D80A380518074803C02066B
:100583002789828A83ECFAE493F5F0A3C8C582C86D
:10059300CCC583CCE493A3C8C582C8CCC583CCB5F2
:1005A300F076DFE3DEE1807089828A83E493F5F0FD
:1005B300A3E208B5F062DFF4805E89828A83E0F506
:1005C300F0A3E608B5F051DFF5804D89828A83E018
:1005D300F5F0A3E208B5F040DFF5803C89828A8319
:1005E300E493F5F0A3E608B5F02EDFF4802A800249
:1005F300805789828A83ECFAE493F5F0A3C8C58215
:10060300C8CCC583CCE0A3C8C582C8CCC583CCB550
:10061300F006DFE4DEE280007FFFB5F0020F224048
:10062300027F012289828A83ECFAE0F5F0A3C8C530
:1006330082C8CCC583CCE0A3C8C582C8CCC583CC53
:10064300B5F0D5DFE5DEE380CF89828A83ECFAE07B
:10065300F5F0A3C8C582C8CCC583CCE493A3C8C5B1
:1006630082C8CCC583CCB5F0AFDFE4DEE280A988D5
:10067300F0EF60010E4E60ABED2402B4040050981D
:10068300F582EB2402B40400508E23234582239089
:10069300056373EF4E6012EF60010EEDBB010B8932
:1006A300828A83F0A3DFFCDEFA2289F05007F70980
:1006B300DFFCA9F022BBFEFCF309DFFCA9F022E872
:1006C3008FF0A4CC8BF0A42CFCE98EF0A42CFC8A34
:1006D300F0EDA42CFCEA8EF0A4CDA8F08BF0A42DB1
:1006E300CC3825F0FDE98FF0A42CCD35F0FCEB8E52
:1006F300F0A4FEA9F0EB8FF0A4CFC5F02ECD39FE08
:10070300E43CFCEAA42DCE35F0FDE43CFC22C3E43A
:100713009FFFE49EFEE49DFDE49CFC22FAE6FB08B9
:1007230008E6F925F0F618E6CA3AF622E557244B0F
:10073300F8E60557227848300702784BE475F00154
:1007430012071F02014C2000EB7F2ED2008018EF0E
:10075300540F2490D43440D4FF30040BEF24BFB49F
:100763001A0050032461FFE55860021558055BE544
:100773005B7002055A30070D7848E475F0011207E3
:100783001FEF0201C50210667403D2078003E4C29F
:1007930007F5578B488A49894AE4F558F55AF55BBA
:1007A300E55860077F2012076A80F57559FFC2017B
:1007B300C200C202C203C205C206C208120738FF42
:1007C300700D3007057F0012077BAF5BAE5A22B472
:1007D300255FC2D5C204120738FF24D0B40A0050E3
:1007E3001A75F00A785830D50508B6FF0106C6A475
:1007F30026F620D5047002D20380D924CFB41A0080
:10080300EF5004C2E5D20402097BD20180C6D200B4
:1008130080C0D20280BCD2D580BAD20580B47F20FA
:1008230012076A2002077401B5580040F112072F1E
:10083300FF12076A0207A3D208D206809512072F78
:10084300FB12072FFA12072FF94A4B7006794C7ADD
:100853000A7BFF20022EE558602A7E008E82758374
:100863000012016560060EEE655970F0C2D5EBC04B
:10087300E0EAC0E0E9C0E0EE1209C2D0E0F9D0E05E
:10088300FAD0E0FB12014CFF60AAEBC0E0EAC0E043
:10089300E9C0E012076AD0E02401F9D0E03400FA9D
:1008A300D0E0FBE5590460DCD559D980877BFF7A1A
:1008B3000979BED202809C791080027908C206C2EF
:1008C300088008D2D5790A8004790AC2D5E559048B
:1008D3007002F559E4FAFDFEFF12072FFC7B082096
:1008E300011312072FFD7B1030000A12072FFE128F
:1008F300072FFF7B20EC3382D592D55013C3E4300E
:1009030000069FFFE49EFEE42001039DFDE49CFCA2
:10091300E4CBF8C201EC700CCFCECDCCE824F8F8D0
:1009230070F38017C3EF33FFEE33FEED33FDEC338B
:10093300FCEB33FB994002FB0FD8E9EB300105F8E0
:10094300D0E0C448B201C0E00AEC4D4E4F78207BA2
:100953000070C2EAB5590040BCC0E01209C4D0F02F
:10096300D0E0200104C4C0E0C4B201C0F0120753B8
:10097300D0F0D5F0EB0207A312045F08405308BA86
:100983005808114C080D4208BE4F08C64408C64912
:1009930008264308CC5508B04608B04508B0470AB6
:1009A3006C5008152D08192E083C2B081D23083AF6
:1009B300200A552A07D548000008343F3F3F0079F5
:1009C3000AA2D5200314300509B910020404B9089A
:1009D3000104A2D52006025001042002689202B548
:1009E30058005034C0E07F203003197F30A20272D8
:1009F300067205500F120A1BC202C206C205C208C4
:100A03007F30800F300503E9C0E012076A30050329
:100A1300D0E0F9D0E0B558CC3005177F30B9100CD1
:100A230012076A7F583004077F788003B9080312DE
:100A3300076A3002057F2D02076A7F202008F87FAE
:100A43002B2006F322920280CF286E756C6C29004E
:100A5300D20112072F3001F8C201785830D50108AE
:100A6300F60207D52D5043495812072F2403B40526
:100A7300004001E4900A679312075B743A12075B24
:100A8300D2037558040208BA30352F32372F303865
:100A93002031393A35353A3532000D0A000D0A490D
:100AA3006E69742E2E2E000D0A253035754B2046A7
:100AB3004C41534820546F74616C0D0A0009253072
:100AC30035754B20464C415348204D656D6F727907
:100AD3002025640D0A000D0A253035754B2046523A
:100AE300414D0D0A002A2A4572726F72212043611B
:100AF3006E6E6F7420636F6E6E65637420746F2007
:100B0300434F4D00436F6E6E656374656420746F6D
:100B130020434F4D002A2A4572726F7221204E6F77
:100B23002064657669636520666F7220434F4D00CC
:100B33002A2A4572726F722120556E7265636F6740
:100B43006E697A656420726573706F6E73652022B7
:100B5300253032582220666F7220434F4D002028E3
:100B6300536174656C6C6974652900202845746849
:100B730065726E6574290054696D657761766520C9
:100B83004453502D443330300D0A4669726D7761FA
:100B930072653A20002052657620332E300D0A53B9
:100BA300657269616C204E756D6265723A2000252D
:100BB3002E3573000D0A0000000020537461727417
:100BC3002E2E2E0D0A0D0A0044535020496E6974CF
:100BD30069616C697A696E672E2E2E0D0A00746541
:100BE3006D7000766F6C747300757074696D650059
:100BF300636F6D316F757400636F6D326F75740061
:100C0300737461747573006C6576656C00676169F4
:100C13006E00766F6C3100766F6C320066726571B0
:100C2300000D0A445350204F66666C696E652E2E84
:100C33002E0D0A007265736574000D0A445350202B
:100C43004F6E6C696E652E2E2E0025642064422043
:100C53005665722025642025630020256420487A88
:100C630000466163746F72792E00476F6F64203A98
:100C73002047756167653A2025753A2575202D3E15
:100C8300200046696C7465726564202D3E20004225
:100C93006164203A20005061636B65743A2025300B
:100CA3003258202530325820253032582025303212
:100CB300580D0A0044697361626C656420445350A3
:100CC3002E2E2E0D0A005772697465204661696CD9
:100CD3007572650D0A002E0069666C6F7773257552
:100CE300003D256C750D00536174205265616420CD
:100CF3004572726F720D0A004D4520526561642082
:100D03004572726F720D0A00FF0A8BFF0A9DFF0C7A
:100D130037FF0CC98B3D8A3E893FAB3DAA3EA93FB5
:100D230012014CFF12002E500D7401253FF53FE4D4
:100D3300353EF53E80E4D200AB3DAA3EA93F120109
:100D43004CFF642B6004EFB42D1BAB3D053FE53F27
:100D5300AA3E7002053E14F912014C642D6003D3C0
:100D63008001C39200E4F543F542F541F540AB3D04
:100D7300AA3EA93F12014CFF12108D505CE47F0A7A
:100D8300FEFDFCAB43AA42A941A8401206C2C8EC2F
:100D9300C8EDC0E0EEC0E0EFC0E0AB3DAA3EA93F26
:100DA30012014CFF3395E0FEEF24D0FFEE34FFFE3B
:100DB300E4FCFDD0E0FBD0E0FAD0E0F9EB2FF54303
:100DC300EA3EF542ED39F541EC38F5407401253F33
:100DD300F53FE4353EF53E809530000AAF43AE4221
:100DE300AD41AC40800BAF43AE42AD41AC401207C6
:100DF3001122434F4D003A20426175642000333085
:100E03003000363030003132303000323430300090
:100E13003438303000393630300031393230300038
:100E230033383430300035373630300025303258DF
:100E33002064656661756C74000D0A0052657072FA
:100E43006F6772616D696E672E2E2E2020253036F6
:100E53006C5800203D205B25303258253032582510
:100E63003032585D0D0A0043616E6E6F74207265F7
:100E730070726F6772616D2E2020496E76616C69A6
:100E83006420646174612066696C652E205B253083
:100E93003258202530325820253032585D0D0A0053
:100EA3008B3D8A3E893FAB3DAA3EA93F12014CFFD1
:100EB30012002E500D7401253FF53FE4353EF53EFB
:100EC30080E4D200AB3DAA3EA93F12014CFF642B44
:100ED3006004EFB42D1BAB3D053FE53FAA3E700216
:100EE300053E14F912014C642D6003D38001C392B3
:100EF30000E4F540F541AB3DAA3EA93F12014CFF8A
:100F030012108D5036AB3DAA3EA93F12014CFF3360
:100F130095E0FEEF24D0FBEE34FFFAAE40AF417C08
:100F2300007D0A1201F9EF2BF541EE3AF540740109
:100F3300253FF53FE4353EF53E80BB300006AE402D
:100F4300AF418009C3E49541FFE49540FE2202309E
:100F53002EE493A3F8E493A34003F68001F208DFA1
:100F6300F48029E493A3F85407240CC8C333C4546E
:100F73000F4420C8834004F456800146F6DFE48022
:100F83000B010204081020408090102FE47E01938F
:100F930060BCA3FF543F30E509541FFEE493A360F4
:100FA300010ECF54C025E060A840B8E493A3FAE44F
:100FB30093A3F8E493A3C8C582C8CAC583CAF0A3A0
:100FC300C8C582C8CAC583CADFE9DEE780BE787EAA
:100FD300E4F6D8FD75818A020F8C8B2E8A2F893017
:100FE300E4F536F537E5351535AE34700215344E74
:100FF3006033AB31AA32A93312014CFFAB2EAA2FB7
:10100300A9300537E537AC367002053614F5828C06
:1010130083EF1201D7EF60CD74012533F533E43547
:1010230032F53280C0AB2EAA2FA93022C18BC18CDE
:1010330000C10E41000000026800000266000004C7
:101043006A00000000017200017C00026F00004191
:1010530005BB004105EF00011500420401000041FA
:1010630005DA00EFB40A07740D121071740A309890
:1010730011A899B8130CC2983098FDA899C298B8D2
:1010830011F63099FDC299F59922EFC394304007C8
:10109300EF943A50028001C32212011001000000B4
:1010A30040C4100480000002030101090220000172
:1010B3000100800F09040000020000000007058101
:1010C30003400005070502034000050705840340AC
:1010D30000051C0309040908090C0910091409185F
:1010E300091C090C09240928092C093009341203A5
:1010F300540049004D00450057004100560045008B
:1011030000000A0344003300300030000000900860
:101113008EE07010A3E0700C900892E07006A3E0DC
:1011230064026002517C90088CE0247F6015146097
:101133002D2402600221BA900890E0707AA3E06047
:1011430015807490089BE0B4040A900890E0700442
:10115300A3E06002806190089812004680509008D6
:101163009BE0B40406900890E06002804A900891E6
:10117300E0FFB48111E56B900898B40304517180CA
:10118300031200468028EFB40211E56C900898B46E
:101193000304517180031200468013EFB48416E5F3
:1011A3006D900898B4030451718003120046D15C1A
:1011B3007402F080048000517CE56A64046007E5F2
:1011C3009620E7FBD1A822F1C26002415E90088C11
:1011D300E0FF7002415E64017002415E90088EE0A0
:1011E3007079900890E07073900892E0706DA3E0BE
:1011F3006002806790088CE06402705F90088FE063
:101203007059F1D0600AEF64026005EF6484704B9B
:10121300EFB48112E59620E7FBF1C9E59620E7FBE1
:10122300D1B9F56B8037EFB4021BE59620E7FB7568
:10123300960E759702E59620E7FB759614759780D1
:10124300E4F56C8018E59620E7FB75960E75970418
:10125300E59620E7FBD1B9F56D8002517CE5962038
:10126300E7FBF1D86007E59620E7FBD1F52274FF91
:10127300F0A37400F0A3741E22E59620E7FB759695
:101283000EE4F597E59620E7FB75961175972075A3
:101293006A042290088EE024FE60221460401470D9
:1012A300026178147002618A2404600261E491335C
:1012B300A37410F0A3749CF090109C61859133A3E8
:1012C3007410F0A374AEF09010B1E493FE9010B0DC
:1012D300E4937C002400FFEC3E90089661DE9008C6
:1012E3008FE014600A14605614605F2403806775EE
:1012F300610274A82561F582E43408F583E0FFE513
:101303006125E02416F582E43408F583EFF0E56106
:1013130025E02417F582E43408F583E4F00561E55C
:1013230061B408CE900818740CF0A37403F090080D
:10133300987401F0A37408F0A37418F08022913319
:10134300A37410F0A374F1F080169133A37411F019
:10135300A37405F0800A9133A37410F0A374D5F03D
:10136300900898E0FBA3E0FAA3E0F912014CFF9088
:101373000896E480669133A37410F0A374B7F090D9
:1013830010B7D155E4805490088FE0FF6481600A60
:10139300EF64026005EF64847047EFB48112913308
:1013A300A37410F0A374C0F09010C0D155E4802B47
:1013B30090088FE0900898B4021074FFF0A37410A3
:1013C300F0A374C7F09010C7800E74FFF0A37410DD
:1013D300F0A374CEF09010CED155E4F0A3EFF080DB
:1013E30002517C90088EE0FF64016013EF64026099
:1013F3000EEF64036009EF64046004EFB405239007
:101403000893E0FFD3900897E09F900896E094003C
:101413004010900892E0700AE0FE900896EEF0A368
:10142300EFF0E56A64046007E59620E7FBD1A822A4
:1014330090089874FFF022E59620E7FB75960EE47A
:10144300F597E59620E7FB759691E59620E7FB85F2
:10145300975FE56AB40511E59620E7FBE4F59690FE
:10146300088FE0F597E4F56AE55F30E20EE5962034
:10147300E7FB759611E4F597F56A22E55F30E41909
:10148300E59620E7FB759611759708E59620E7FB2F
:10149300759611759780E4F56AE56A6002A14AE5DD
:1014A3005F20E002A14A7B017A08798C7D087C00E9
:1014B3007F201240DD90088FE0FE90088EE07C00D4
:1014C3002400FFEC3EF0A3EFF0900891E0FE9008BB
:1014D30090E02400FFEC3EF0A3EFF0900893E0FED1
:1014E300900892E02400FFEC3EF0A3EFF090088D0B
:1014F300E0B40C00504F901500F82828730215240F
:1015030002152802154802152C021548021530024F
:10151300153402154802153802153C021540021510
:10152300443111802231CA801EF1E3801AD1FC803C
:101533001651968012D101800EF143800AD1648046
:1015430006D1C18002517CE56A64016002C100E5F5
:101553005F30E102C100E59620E7FB759691E596C1
:1015630020E7FB85975FE55F30E40530E002C100CB
:10157300756002C3900897E09440900896E0940049
:10158300403C900898E0FBA3E0FAA3E0F97D407C9F
:10159300007F20124027900899E475F04012026002
:1015A300900897E024C0F0900896E034FFF090088C
:1015B30095E02440F0900894E03400F0801C9008FB
:1015C30096E0FCA3E0FDA3E0FBA3E0FAA3E0F97F30
:1015D30020124027436008E4F56A900892E0FEA3D6
:1015E300E0FFA3E0B5060BA3E0B50706436008E4FC
:1015F300F56AE59620E7FB759611856097229008BA
:101603008CE06480701C90088EE07016A3E070126A
:10161300A3E0700EA3E0700AA3E07006A3E06401E8
:101623006004517C801E90089BE0FFB40408913352
:101633005174D15C04F0EFB4030A90089812004689
:10164300D15C04F0E56A64046007E59620E7FBD10A
:10165300A822E493FF90089622F0900896E4F0A362
:1016630022F1C2702490088CE06481701C90088E73
:10167300E07016A3E07012A3E0700EA3E0700AA35B
:10168300E07006A3E064016004517C800A9008982E
:10169300120046D15C04F0E56A64046007E5962015
:1016A300E7FBD1A822759611759740756A01E490FE
:1016B3000894F0A3F022759611759740E4229008E0
:1016C3008CE06401701C900892E07016A3E0701225
:1016D30090088EE0700CA3E07008A3E07004A3E010
:1016E3006002517CE56A64046007E59620E7FBD15C
:1016F300F5227596117597482290088CE0701D901D
:101703000890E07017A3E07013A3E0700FA3E070DC
:101713000B90088EE07005A3E030E702517C756AF8
:101723000590088FE090089B60057403F0800374B4
:1017330002F0E56A64046007E59620E7FBD1F52231
:1017430090089BE06402602590088CE0701F90086D
:1017530090E07019A3E07015A3E07011A3E0700D81
:1017630090088EE07007A3E0D394014004517C807D
:101773004090088FE0D39400402D90089B7404F0B0
:10178300E4F56BF56CE59620E7FBF1C9E59620E7F8
:10179300FB759612759720123FC4E59620E7FB75FB
:1017A300960EE4F597800A90089B7403F0F56BF5A9
:1017B3006CE56A64046007E59620E7FBD1F52290A7
:1017C300089BE064042275960E7597012290089198
:1017D300E0FF64812275960EE4F597E56A640422BE
:1017E300F1C2600302188A90088CE0FF70030218AC
:1017F3008A6401700302188A90088EE06002018AED
:10180300900890E06002018A900892E07079A3E06A
:101813006002807390088CE06402706B90088FE024
:1018230070651217D0600AEF64026005EF6484707C
:1018330056EFB48118E59620E7FB1217C9E5962009
:10184300E7FB759611759710756B03803DEFB40236
:101853001BE59620E7FB75960E759702E59620E744
:10186300FB759614759720756C03801EE59620E72B
:10187300FB75960E759704E59620E7FB7596117533
:101883009710756D03800312127CE59620E7FB1217
:1018930017D86008E59620E7FB1216F522F1C7E496
:1018A300F526E4F525AF25122844122FB3E475502D
:1018B30001F54FF54EF54D7F90122F361200268F0E
:1018C300231200268F24E52312045F19044118F51F
:1018D3004318FA4418FA4818ED4918FF8018FA8D8E
:1018E30018FF8E190CFF0000190C7527007528804E
:1018F300801C752701800D752702800875270480D9
:10190300037527087528008005E4F527F528D3E536
:10191300289400E5279400400EAF251245B1AF256A
:101923001228447F013196E52525E0249CF582E4C5
:101933003408F583E527F0A3E528F0124561E4F0C8
:10194300A3F0AF25EFD39400401DEF25E0249AF5D3
:1019530082E43408F583E0FCA3E0FD124561EC8DDD
:10196300F01202601F80DD0525E525C394035002B4
:1019730001A8F1C70526E526C39402500C9008A4DC
:10198300E07002A3E0700201A52212311DE4FF31D1
:101993009AE4FF319AE4FF30F9FDC2FF8FA330FFD1
:1019A300FD2290058DE0FDE4FF8F318D32741D2FF4
:1019B300F8E67002FF22F1C7AF31318DAF3112313A
:1019C3001D7FA3319A0000000000AF321227968FCB
:1019D30032F1C7E5327003123164E532700312311C
:1019E30064AF32227E007A05797B1244E67A057968
:1019F3003B1244E67F0E7D007B017A0579BC12061B
:101A0300967E007F107D007B017A0579CA120696C7
:101A1300E47871F6787412044600000000787812B6
:101A2300044600000000E4900539F0A3F07BFF7A40
:101A33000A79A01222901222827FFF7873EFF612A6
:101A43004139787D7602122FEC8E4E8F4F754BFF06
:101A5300754C0A754DAAF1A8122290F1B11227AF65
:101A6300123984E4F516754BFF754C0A754DC0E5C4
:101A73001625E0249CF582E43408F5831245C9E574
:101A8300162401F551E433F550F1A8122290F1B177
:101A93001227AF0516E516C3940340CA1239841200
:101AA30037E7754E008F4F754BFF754C0A754DD94F
:101AB300F1A8122290F1B11227AFE4F517E4F5165D
:101AC3001245E8BFFF091245E8EFF4600580007591
:101AD3001601E5167010741D2517F8E670057516C6
:101AE300028003751603E516146012146017146060
:101AF3001C2403702C7BFF7A0A79E880217BFF7A10
:101B03000B790780197BFF7A0B79188011754BFFCE
:101B1300754C0B754D33754E0085184FF1A8122285
:101B230090E5172432FF123C74E51714600B047020
:101B3300117BFF7A0B796180067BFF7A0B796E123A
:101B430022907BFF7A0A799D1222900517E517D31D
:101B53009401500241C012445C900541E0FF123CE5
:101B6300C6AD077F01122338900542E0FDE4FF3143
:101B7300ACAD077F021223387D257F0131ACAD0761
:101B83007F03122338123EAB123984C2901241F004
:101B9300C20AC209D28290055674FFF01245587BDF
:101BA300FF7A0B797A122290900D0B1222857BFF1C
:101BB3007A0B7998122290754BFF754C0B754DB2C9
:101BC300754E01754F087550AAF1A81222907A0B31
:101BD30079B712397F7A0B79BD12397F30820A12B5
:101BE30044BF7A0B79CB1245D1123984123EAB78BC
:101BF300841203F578741245E1503278841203F5A8
:101C0300EF24191226E5787412042E7882E6FE0872
:101C1300E6FF7C007D0B1201F99005C6EEF0A3EF01
:101C2300F07880E6FF08E6A3CFF0A3EFF078841204
:101C330003F578781245E14002A1F778841203F5A1
:101C4300EF24F4FFEE34011226E8787812042E789C
:101C53007C06E6C39402405DE4F67872069005D6EE
:101C63001223E324011226E59005D61245C130E480
:101C730008787006E6187001061245D94003E0049F
:101C8300F09005EFE0D394004010E004F0D3940A01
:101C93004008787DE654FEF6E4F0300E1290000022
:101CA300E0D394004005E014F0800AC20E80069051
:101CB3000000740AF0309104C2918002D291900521
:101CC30043E020E402A1D890057BE030E102A1D8F3
:101CD300AF150515EF12045F1D18011D23021D2EFC
:101CE300031D39041D65051D44061D65081D5A0A9B
:101CF3001D650B1D730C1D650E1D65101D65121DE5
:101D03005A141D65151D73161D80171D8D181D98FA
:101D13001B00001DAB7BFF7A0B79E19005C8807E29
:101D23007BFF7A0B79E69005C680737BFF7A0B798C
:101D3300EC9005D680147BFF7A0B79F39005CA806B
:101D4300097BFF7A0B79FB9005CE1223E3F5478ECF
:101D5300468D458C44804A7A0C7903900543F1D033
:101D6300803F7BFF7A0C790A90053F124549803109
:101D73007BFF7A0C79109005BCF1D280247BFF7A2B
:101D83000C79159005BEF1D280177A0C791A90055B
:101D9300BFF1D0800C7BFF7A0C791F900539124577
:101DA300497F01124350802DE515C3941C4003E481
:101DB300F515900401E0FEA3E0FF12431590040221
:101DC300E02408F0900401E03400F0C3E0942040E4
:101DD30004E4F0A3F0D37870E694B418E6940040DA
:101DE3001FE4F608F6124598F07B107D107F011270
:101DF300384A800CF1B17DFF12257EF1B1123BA967
:101E03007973E7787D6670051245D9403A9005BB32
:101E1300E0FFD394004026EF75F00684AFF0740121
:101E2300A807088002C333D8FCFF1241399005BBD1
:101E3300E0C3943C4011E4F07873F6800A787DE6C1
:101E43007873F6FF12413920821090053DE0440477
:101E5300F0F1B17DFF122016800D1244BF300A0746
:101E63007A0C79241245D1F1B17DFF1228D4F1B156
:101E7300123BA9123EF5400261F2123E8E8F16E527
:101E830016C394005002E13390040BE516F0E4A36B
:101E9300F078037C047D017B017A047904FE7F07DB
:101EA300120126900409E516F0E4A3F0F1B1122221
:101EB3009078057C047D01900D11E4124525F97E8F
:101EC300007F05120672EF600261F2900D11124558
:101ED30025F9E4754701F1D77F011243507F007E56
:101EE300007D047C001227F21243BC9005DFE4F06E
:101EF300A3740CF09005DDE4F0A3740CF09005E1FD
:101F0300E4F0A3740EF09005E7E4F0A37480F0907E
:101F130005E5E4F0A37480F0E4A3F0A3F0A3F0A339
:101F23007483F0A37401F0A3742CF0122E6C61F28D
:101F3300E4FFAD07900796E0C394CE4004F1F5802B
:101F4300F3E4FF8D28123E9A752901F52A892BF1B6
:101F5300F51245429001A5120165C394CE4002D308
:101F630022C2AC1245429001A3120165FF7E00E933
:101F730024D0F9E43AFAE92FF9EE3AFAE5281245C2
:101F83003F9001A37401120192E924A3123E0F12A0
:101F93003DAC12453F9001A57401120192123E0C13
:101FA300123E92C3227B017A04790B12078B7B01C9
:101FB3007A04790B2253903B43A03DD2954390443E
:101FC3007F06319A53903B43A03DD295227BFFE09D
:101FD300FFE48F47F546F545F54422741D2FF8E6D7
:101FE3007002FF22F1C712311D7FA5319A12279982
:101FF30080D2900797E030E00554FEF0D299227F1B
:10200300031245B17F031228447F0112199AE4FF9A
:1020130002199AF1A8E4FD300A0201EA7BFF7A0C67
:10202300793D5190D20A30090201E01231AD12001C
:10203300181102122E8612387C754BFF754C0C75E5
:102043004D4D9005BCE024E8F54FE434FFF54E9088
:10205300088812459F7F4430E1027F508F527131CF
:1020630012078B713151907D1A7F011235EE7D1A63
:102073007F02123692123687F0E4F519F51AF54607
:10208300F545754404F5437A007927F5477548000B
:10209300754927F1EA754601754500754404754392
:1020A300007A007926754700754800754926F1EADC
:1020B300C3E52794A0E526940F502A754BFF754C72
:1020C3000C754D5DAE26AF27900539EEF0A3EFF00A
:1020D3008E4EF54F713112078B713180067BFF7A7B
:1020E3000C7964519051823009024181E51A75F0EF
:1020F3001484E5F0702612387C900889E090053D41
:1021030030E006E04408F08004E054F7F0900886DD
:10211300E0FFA3E090053FCFF0A3EFF0051AE51A27
:10212300D394C850024181E4F51A90087DE09005EC
:1021330044F0E070024181E51954F0FFE054F06F80
:10214300603653190FE054F04219E51954F0C454A2
:102153000FF526787DE654E3F6E526D3940C400686
:10216300E64410F68012E526D39409787DE640050F
:102173004408F680034404F6E519540FFF90054420
:10218300E0540F6F700241815319F0E0540F42196C
:102193007B017A057945123766900545E0FF121FEA
:1021A30035900546E0FF121F35900547E0FF121FEB
:1021B30035900548E0FF121F359005CA71E3D1E35E
:1021C3009005CA12043A752B01752C05752D0A7BEF
:1021D300017A05794512340CEF6053787DE64401AA
:1021E300F69005EF7401F0754BFF754C0C754D6D52
:1021F30090050A1245C9A3E0F550A3E0F5517131EA
:1022030012078B713151901245A812442BEF7007BE
:10221300900543E030E70D1245A8A3E0FCA3E0FDE1
:1022230071EE802F7BFF7A0C7985519080251244C3
:10223300C67BFF7A0C79925190900543E030E71307
:10224300B174E4FFB1069005CE71E3D1E39005CEFE
:1022530012043A754BFF754C0C754D99900545E08A
:10226300754E00F54FA312459F755200F553A3E039
:10227300755400F555713112078B713151902290CD
:102283000D0EE493FB740193FA740293F98B468A5F
:10229300478948EA494B60141200038E498F4AABC1
:1022A30046AA47A948AD4AAC49123A2AE5C930E6DD
:1022B3006590057FE0FF900554E06F70591239FE79
:1022C3008E498F4AD3E54A9409E54994004006753F
:1022D3004900754A09D3E54A9400E5499400403121
:1022E30090053DE04401F07B017A05794AAD4A123D
:1022F3003AEC900555E54AF090057FE0C3947E5093
:1023030008E004900554F0800D9005547401F080AA
:1023130005E4900555F090053DE054FEF022122EA1
:10232300EE900585E0FF7E00788D7C057D01AB2373
:10233300AA24A925228F2E8D2F7BFF7A0D79F551A3
:1023430090E52E2430FF123C747BFF7A0D79F9510E
:1023530090E52F12045F237801238002238804234E
:10236300900923981223A02523A84B23B09623B8C2
:10237300E1000023C07BFF7A0E790180567BFF7A50
:102383000E7905804E7BFF7A0E790980467BFF7AB2
:102393000E790E803E7BFF7A0E791380367BFF7AAF
:1023A3000E7918802E7BFF7A0E791D80267BFF7AAB
:1023B3000E7923801E7BFF7A0E79298016754BFFD9
:1023C300754C0E754D2F754E00852F4FD1DC1207BE
:1023D3008BD1DC51907BFF7A0E793C419090058143
:1023E300E0FCA3E0FDA3E0FEA3E0228E288F298C6E
:1023F3002A8D2B53281F532A07900543E030E147CA
:10240300EF543F44C0F52CE529AE287806CEC3131C
:10241300CE13D8F9547FFFAE2BEEC433333354803D
:102423004FF52DE52AC313E52B13F52EE52AC31328
:102433005403F52F7B007A00792C1243CA8F30E5C1
:102443003054FC422F8079D3E5299463E528940026
:102453004042E529543F4440F52CE529AE2878064F
:10246300CEC313CE13D8F9543F4440F52DE528C409
:102473005401FFAE2BEE25E0543E4F44C0F52EE54C
:102483002BAE2A7805CEC313CE13D8F9543F44C0DC
:10249300F52F802CAE28AF29B15CEF540F4403F520
:1024A3002CAE28AF29B15CED540F4403F52DB15880
:1024B300EF540F4403F52EB158ED540F4403F52F99
:1024C3009005421219A87B007A00792C754C04E41C
:1024D300FFB1069005CE71E3D1E39005CE1245C15D
:1024E30030E41D7530ABD1DC754C01B163B1637F52
:1024F30001B1069005D271E3D1E39005D212043AFB
:102503007F01228B498A4A894B741D2FF8E6604468
:10251300121FC712311D7F5A12199A0000000000C2
:102523007F0112199A0000000000AF4C801EAF4CCF
:10253300154CEF601C0000000000AB49054BE54B58
:10254300AA4A7002054A14F912014CFF12199A8023
:10255300DD121FC722AE2AAF2B7C007D0A02020BBD
:102563007F01B1067B017A057945754C047F01B182
:10257300067B017A057945754C0422F1A88D26E482
:10258300F5277F01121FDE8F2AE52AB4FF087BFFA0
:102593007A0C79FBC1CEE52A7002C1D0E52A541822
:1025A30064086002C1DB7131E52614F52F7F01F168
:1025B300328F28E528D394005002C1C571311237F8
:1025C300CD9005DAE0D394004005E4F529C185E414
:1025D300F529E529C395284002C1C57131852982B2
:1025E300758300120165F52A54F0FFBFF0178528A3
:1025F30041AD291236188F28E52A64F66007900545
:1026030043E04410F0E52A240CB40B004002C1C19E
:1026130090261A12456F730226B50226AD02264490
:1026230002268502267C02267302266902265F02A1
:10263300265602264D02263B900543E01245B980FB
:1026430091900543E054EFF08088900543E0440106
:10265300F0A1D5900543E054FEF0A1D5E4786FF6E0
:1026630008F6D290A1D5E4786FF608F6C290A1D50A
:10267300900543E04420F0A1D5900543E054DFF0FA
:10268300A1D5C3E5289529F528AB237E00E52525AB
:1026930029F9EE3524FA752E00752F0075302812AE
:1026A30031F8E5292528F528A1D5900543E0440212
:1026B3008006900543E054FDF0122F66A1D505294D
:1026C300A1D5E528D394004004713151900527E545
:1026D30027C3940A5002A185227B007A0079302215
:1026E3002404FFE43EFEE43DFDE43CFC22F1A88D1E
:1026F30026E4FF121FDE8F27E527B4FF087BFF7A4E
:102703000C79EA8027E5276025E5275418640870CB
:102713001D7131E52614F52FE4FFF1328F1C713161
:102723001237CDE51CD39400400471315190228BB4
:102733002C8A2D892E741D2FF8E67003FEFF2212BA
:102743001FC712311D7F5512199A7F01F1968F30E1
:10275300E530D394004034E4F531E531C39530508E
:102763001DE531C3952F5016F199AB2CAA2DA92E37
:10277300853182758300EF1201D7053180DCE531A5
:10278300C395305006F199053180F3121FC7AF305E
:102793007E002212199AE4FF000FBF96FBE4FF129A
:1027A300199AAFA3228B238A24892522F1A89007A3
:1027B30096E0700E1200038F267131EFFD7C00024C
:1027C3003E17713112014C601D713112014CFF1221
:1027D3001F355005121FF580F074012525F525E4FA
:1027E3003524F52480DC22754A017F03022EEE8F07
:1027F300438E428D418C408F488E478D468C457F5A
:10280300038004F5457F028F44114400000000005B
:102813007F0612199AAF4411440000000000854856
:102823005085474F85464E85454D7F20F136539061
:102833003B43A03DD295F1B3AF44D128EF20E0F85C
:102843002253903B43A03DD295EF146011146012C4
:10285300146013146014240470134390842243906F
:1028630080224390C02243904022439044228F40D1
:10287300854849AF481548EF604CAF40114400000C
:102883000000007F0612199AAF40114400000000B7
:1028930000784112040E8F508E4F8D4E8C4D7F0267
:1028A300F1360000000000AB450547E547AA467036
:1028B30002054614F912014CFF12199AAF40D128B0
:1028C300EF20E0F880AD53903B43A03DD295AF4954
:1028D300221227A8E4FD90057DE0FF900549E06FF3
:1028E300700241C290057CE024D0700241B1242FD4
:1028F300B41800400241BF90290112456F730229A9
:1029030054022ABF02296C0229760229D40229D94A
:10291300022A170229810229930229600229CA0285
:1029230029F20229A50229B7022ABF022A4D022948
:10293300490229660229E3022A35022AA9022A0743
:10294300022A89022A97E4900558F0900556F0412F
:10295300BFD1207F01D14FD1207F02806ED1207F54
:10296300078068D1207F09806290058DE0FD1236D3
:1029730090805A90058DE0FD123683F0804FF19ED2
:102983007F05D14F9005C2E0FCA3E0FD7F06803BAD
:102993009005C0E0FCA3E0FD7F05D14FF19E7F06CB
:1029A300802990058DE0FF123CC6900541EFF0FDB4
:1029B3007F01800E1219A51219A5900542EFF0FDB3
:1029C3007F021223388006F19E7F08D14FF16641C2
:1029D300BF1241F041BF124598F07B107D10800873
:1029E300124598F07B307D307F0112384A41BF9009
:1029F300058DE09005436006E04480F041BFE0545C
:102A03007FF041BF900888E0900559F09005577416
:102A130001F041BF12455890057C7411F0F166E452
:102A2300F526F1B30526E526C3946440F543EF90FC
:102A330041BF90058DE06009D20943A404C282809E
:102A43007BC209D28253A4FB80727B017A05798D04
:102A5300900586E0F54C7F011225069005D2E0F83B
:102A6300A3E0F9A3E0FAA3E0FB900586E0FFE4FC12
:102A7300FDFEEB2FFFEE3AFEED39FDEC38FC900541
:102A8300D212043A80367A0579BC7F0E1244F212D0
:102A930045B980287A0579CA7F101244F254EFF0C1
:102AA300E04420F080169005BBE004F0800E122372
:102AB300317F007E107D007C001238CF1245589084
:102AC300058BE0FF900558E06F700261B0E4FFFEF4
:102AD3007D10900587B1EA402C308212900558E0B2
:102AE30064FE700261B012458E12229061B09005AF
:102AF300871223E3B1FA12457AF1A78526431244DC
:102B0300D27F03619E7FFF7EFF7D0F7C0090058750
:102B1300B1EB7020900D0B1245258B318A32F533C2
:102B230090058CE0753400F5357B017A05795912EF
:102B33000FDD8069E4FFFE7D0FFC900587B1EB405C
:102B43001D9005871223E3F1C2E527940FD11112DB
:102B530045157A05795990058C1237D6803FE4FFE5
:102B6300FE7D0EFC900587B1EB403C900587122358
:102B7300E3F1C2E527940ED111F528E4F527F526F4
:102B83002529F529E5283410F528E43527F527E428
:102B93003526F1A7F5431244D27F02D1EE90058B7F
:102BA300E0900558F0800690055874FDF090057E7E
:102BB300E0FF900556E06F7002A1E4E47D10B1E5FB
:102BC300407D308210900556E064FE7002A1E4124D
:102BD300458E0222901223E0B1FA12457AF526E5DA
:102BE30029FFE528540FFEE4FDFCEE4F7011F51BA1
:102BF3008F488528478527468526457F03110A1276
:102C030045044006122282E4F51B852944852843A6
:102C1300852742852641F1DE900585E0F5487F034F
:102C23001171F1A985264312452F7F031223211227
:102C33000672EF7002A1CE900D14122285A1CEE48C
:102C43007D0FB1E5403C1223E0F1C2E527940FD19B
:102C5300111245157A05798D900585E0754200F5C9
:102C6300431237EFAE28AF2912233190058512376F
:102C7300D6122324120672EF6006900D14122285D9
:102C8300A1CEE4FFFE7D0EB1E75002A1D71223E0EF
:102C9300F52D8E2C8D2B8C2A9400F52DE52C94008C
:102CA300F52CE52B940EF52BE52A9400F52AE52D5A
:102CB300F52DE52CF52CE4F52BF52A252DF52DE541
:102CC3002C3410F52CE4352BF52BE4352AF52A1298
:102CD3004584FDFCEE4F7011F51B8F48852C47850D
:102CE3002B46852A457F02110AE4FB7A10F9F8AFD7
:102CF3002DAE2CAD2BAC2A1203298E268F279005DF
:102D030085E0FFEF252DFFE4352CFEE4352BFDE4B4
:102D1300352AFCE4FB7A10F9F81203298E288F294F
:102D2300E52765297004E52665286065124584C397
:102D33009FF52774109EF526900585E0C39527F52A
:102D430029E49526F5288F44F1D58527487F02117C
:102D530071E527252DF548E526352CF547E4352B78
:102D6300F546E4352A1106E527252DF544E52635F4
:102D73002CF543E4352BF542E4352AF541748D25D2
:102D830027F9E43405754501F546894785294880C7
:102D93000B852D44F1D5900585E0F5487F0211712F
:102DA3001245044006122282E4F51B852D46852C2C
:102DB30045852B44852A4312452F7F021223211276
:102DC3000672EF6006900D1412228590057EE09046
:102DD3000556F022E4FFFE7D0DB1E790055674FD24
:102DE300F022FFFE900581FCE0F8A3E0F9A3E0FAEE
:102DF300A3E0FBC30203D1F5298E288D278C26C3BC
:102E03009400F529E5289400F528E5279410F52783
:102E1300E5269400F526E529F529E5282290058D78
:102E2300E0FD7C00228F4A114400000000007F0572
:102E330012199A00000000001200268F4A53903B9B
:102E430043A03DD295AF4A22AC39AD3A8F3D8C3E7B
:102E53008D3F1243BCE53D25E024DBF582E43405D8
:102E6300F583E53EF0A3E53FF0E4F544F543754211
:102E730005F5417545017546057547DB7548147FB2
:102E8300031171D1D69005DEE09005BCF09005E208
:102E9300E09005BDF09005E5E0FFA3E09005C0CF0D
:102EA300F0A3EFF09005E7E0FFA3E09005C2CFF0B9
:102EB300A3EFF09005EAE090053BF09005EBE0FF0F
:102EC300A3E09005C4CFF0A3EFF09005EEE09005EA
:102ED3003CF022E4F546F545754405F54375470195
:102EE3007548057549DB754A147F031144000000DA
:102EF300000085465085454F85444E85434D7F03ED
:102F0300F136854A4BAF4A154AEF601C00000000BA
:102F130000120026AB470549E549AA487002054857
:102F230014F9EF1201C580DD53903B43A03DD295C8
:102F3300AF4B2212199AAF50AE4FAD4EAC4D8F54DA
:102F43008E538D528C5178101203E212199AAF549A
:102F5300AE53AD52AC5178081203E212199AAF5432
:102F630002199A7B017A05793B754200754340E467
:102F7300FFFE1237EFE4F548F547F5461106E4F591
:102F830044F543F542F5417A05793B7545017546AC
:102F93000575473B7548407F02017190058DE0FC44
:102FA300A3E0FD22F5268529468528458527442269
:102FB300E4FFFE0FBF00010EBE01F8BFF4F522F5DA
:102FC300298E288D278C269400F529E5289400F571
:102FD3002822852C43852B42852A417A05798D75D4
:102FE300450175460575478D229008A0E0FEA3E0D4
:102FF300FF22121FC74390447F0512316BEF700409
:10300300C20B80241200268F23E523B4FF04C20BD6
:103013008016121FB84390445323F953237F7F0133
:1030230012199AAF2312199A021FC753D9BF759069
:103033000312414F53903B43A03DD2951241871257
:1030430041774380041242301242A1123C8212188B
:10305300A0122FF511B5E51D6004E51E700211B530
:103063007B017A0879AA7545007546057F007E01C4
:10307300F10975220274A82522F582E43408F58348
:10308300E0FFD3947F5006EFC3942050117E007F5E
:10309300057D307B017A0879AA12069680070522FE
:1030A300E522B407D0E49008AFF0A3F01241A502E3
:1030B30019E7121FC7E4F524E4F523122FB3AF2356
:1030C300311D7FA5316BEF7009741D2523F8E4F6DC
:1030D300800C1227998F25741D2523F87601741D02
:1030E3002523F8E66016AF23311D4325017FAA127D
:1030F300199A0000000000AF2512199A0523E52351
:10310300C3940240B6121FC70524E524C39402509A
:1031130008E51D7004E51E609F22121FC7EF1460AF
:1031230007047006C2A48002C2A0E4FFFE000FBF22
:1031330000010EBE03F7BFE8F4228F33741D2FF88E
:10314300E67002FF22121FC7AF3312198DAF33315E
:103153001D00000000007FA412199A122799021F74
:10316300C7AF31313D8F3222E4F528F52930F9FD1F
:10317300C2FF8FA320FF1A0529E52970020528FF46
:10318300AE28E4FCFD7B507AC3F9F8D31203BB509D
:10319300E3AE28AF29E4FCFD7B507AC3F9F8D312E0
:1031A30003BB50037F00227F0122D20C121FC731C1
:1031B300C97F80316BEF7004C20C800731C97FA0D7
:1031C30012199A021FC75390FB43900422200C0349
:1031D3007FFF22121FC731C9BF01047FC080027F56
:1031E300C212199A31C9120026EF541FFFC3741F6C
:1031F3009FFF021FC78B2B8A2C892D910512014C2F
:10320300F53171FA12014CFF603A640D6036910595
:1032130012014CFFD39400402B9005DAE094135035
:103223002371FA12014CFE9005DAE0FD04F07425D7
:103233002DF582E43405F583EEF08F419101EF1211
:1032430001C580BE9005DAE07011E0FF04F074253B
:103253002FF582E43405F5837420F09005DAE0D38A
:10326300941340037413F09005DAE02425F582E407
:103273003405F583E4F0E531D39400400971FA1283
:10328300014C640D600B71FA12014C640A60026117
:10329300EAE49005DAF0910512014CF54171FA91D7
:1032A30001EF1201C5D15FB1E712014CFF60086461
:1032B3003D6004B1D280F0EF643D600261EAAB325D
:1032C3000534E534AA337002053314F9E41201C559
:1032D300B1E712014CB42004B1D280F4120D178F60
:1032E3003A8E398D388C37D15FB1E712014CB42057
:1032F30004B1D280F4120EA38E358F36C3E5359414
:10330300205051E5367803CEC313CE13D8F9D175C7
:10331300F103E536F1DE8002C333D8FCF53CAF3A66
:10332300AE39AD38AC37EC4D4E4F7007E53CF45237
:103333003B8004E53C423BE536AE357803CEC31310
:10334300CE13D8F9D175754200754301F1EFAF364D
:10335300AE358047E5368535F012048533A320006A
:1033630033AB2001337B6001338160023388600318
:10337300339A6004000033EAAD3AD1908069AD3AE4
:10338300D183F080627F01122E4B7F02122E4B12EB
:103393002F661241F08050AE39AF3A124315804781
:1033A3007E007F147DFF80067E007F147D007B01FD
:1033B3007A057925120696E4F535F536C3E5359495
:1033C300045024E42536FFE5353402FE7B017A05FB
:1033D3007925754200754314F1EF74142536F536DB
:1033E300E43535F53580D5910512014C71FAF58236
:1033F300758300E40201D7AB2BAA2CA92D22E4FD8F
:10340300D118AB2EAA2FA930228B288A29892A7199
:10341300FA74FFF5F01202A171FA90000274FFF53D
:10342300F01202C09161124415EF4E60079158B13A
:10343300017F01229161D19EEF4E600791589168FF
:103443007F01229161D1CCEF4E60079158B1987FF3
:1034530001227F0022852B31852C32852D33AB2829
:10346300AA29A92A228B2E8A2F8930B1925401C40A
:1034730054F091FA75F00091F7C003C002C0011235
:103483000276FDACF09105D16F7E00543F7806C300
:1034930033CE33CED8F9D157D001D002D00391F433
:1034A300C003C002C001120276FF9105F1B2D00140
:1034B300D002D003F1AB9105B192543EFFE4C313A4
:1034C300FEEF13FF91FAF1BCC003C002C001120268
:1034D30076FDACF0B1C67E00543F7805C333CE33DE
:1034E300CED8F9D157D001D002D003EE8FF002022B
:1034F300A1EE8FF01202A1AB31AA32A93322D16916
:103503007E00547F7806C333CE33CED8F9FF91FAC9
:1035130091F4C003C002C001120276FF9105F1B21B
:10352300D001D002D003F1AB900001B1C97E0054A9
:10353300807807CEC313CE13D8F9FF91FAF1BCC03C
:1035430003C002C001120276FD9105B19225E0FF8E
:10355300E43345F0FEED4FFFD001D002D003EE8FF0
:10356300F01202A1AB31E5332402F9E43532FAC09B
:1035730003C002C001120276FDB1C6540325E04523
:10358300F0FFEDD001D002D003CF8FF00202A19063
:103593000002020165D169D14F12014C540F7C0026
:1035A3002FFFEC35F091FA8FF01202A1B1C6D14F83
:1035B300B192540F2FFFEC35F091FA9000028FF087
:1035C3000202C0900003AB2EAA2FA930020165743A
:1035D300012534F534E43533F53322AB32AA33A96C
:1035E3003412078BAB32AA33A934228D3D300C241D
:1035F300121FC7E53D541FFEC3741F9E541FF53DA4
:1036030031C9BF0104AF3D8005E53D4440FF1219B8
:103613009A121FC7228B3D8A3E893F1541EDC39500
:1036230041501BEDF582758300A3AB3DAA3EA93F34
:103633001201658D827583001201D70D80DFAB3DCA
:10364300AA3EA93F854182F1CFAF4122540F75F0C5
:103653000AA4FF22FFEC4EFEED4FFF2275320175E7
:103663003305753425228B2E8A2F89309000010271
:1036730001652400FFEE3402FE7B007A00793B22D1
:103683007F02B1EE7F0231D09005BFEF227F01B1FF
:10369300EE7F0131D09005BEEFF02212014C54C0F1
:1036A30064407021D16F54C064407019B19254C00A
:1036B300FFBFC01190000312016554C0FFBFC005D6
:1036C3007E007F0122E4FEFF2212014C547064301D
:1036D3007021D16F547064307019B1925470FFBF70
:1036E30030119000031201655470FFBF30057E0056
:1036F3007F0122E4FEFF222400FFEE3402FE7B0062
:103703007545007546018B428A438944AD07AC0673
:10371300E4F547F548300B06E54645457004E4FEFD
:10372300FF22121FC74390447F03123838E5461522
:1037330046AE45700215454E601B120026AB42058E
:1037430044E544AA4370020543F1600548E5487027
:1037530002054780D8121FC7AE47AF482214F9EFBE
:103763000201C58B288A29892A90087FE0FF052A50
:10377300E52A70020529F160900881F1A070020525
:1037830029F160900883F1A070020529F160900887
:1037930085F1A07002052914F9EF0201C5E0FFAB22
:1037A30028052AE52AAA2922E5F08FF00202A112B0
:1037B300014C543FFDEF4DFF22900002EE8FF012BB
:1037C30002C0E92402F9E43AFA228F82758300E405
:1037D3000201D7E0754500F546E1095407FF74017E
:1037E300A80708227F08200B027F00228E3D8F3E10
:1037F3008B3F8A408941300B3BE54345426035129C
:103803001FB8439044AD3EAC3D7F021138E54315EC
:1038130043AE42700215424E6017AB3F0541E5418E
:10382300AA407002054014F912014CFF12199A8044
:10383300DC121FC7228C498D4A12199AE549FF12DF
:10384300199AAF4A02199A8F2E8D2F8B30741D2F20
:10385300F8E66024AF2E121FDE8F31AF2E12311D1A
:10386300E52FF45231E53042317FAA12199A000054
:10387300000000AF31121FC522208235121FC7C2BC
:103883009500000000000000000000E4F528AF28C8
:103893007E0011B5E52825E0247CF582E43408F5A3
:1038A30083EEF0A3EFF00528E528C3940840DFD2A8
:1038B3009522AD07AC06AF04EC1227A2AE07AF0505
:1038C3001227A2AD07AF06EFFEEDFF22916B8B32FD
:1038D3008A338934754BFF754C0E754D3F8F518E6E
:1038E300508D4F8C4E1235E412229031E478101231
:1038F30003E28F3F31E478081203E28F40853141C0
:10390300754BFF754C0E754D56754E00853F4F75C3
:1039130050008F517552008541531235DE122290AB
:10392300853146853045852F44852E43754700757F
:103933004800754935754A037F02122EEEE535645A
:10394300026021754BFF754C0E754D6A754E0085EF
:10395300354F7550008536517552008537531235F2
:10396300DE022290E4FFE4FE000EBEFFFB0FBFFF6A
:10397300F53184AB41AD40AF3F02F8007BFF12222B
:1039830090E5C930E63778841203F5EF2432F54524
:10399300E43EF544E43DF543E43CF54231FED3EF28
:1039A3009400EE9400400831ED400471AE80ED3197
:1039B300ED402DE4F566F567F568F56922511EC300
:1039C300EF9420EE94005018C3E49569F543740412
:1039D3009568F542E5692420FFE4717A5002C20E2E
:1039E30022AF31AE30AD2FAC2E2278841203F5AB6B
:1039F30045AA44A943A842D30203D1719F400BE5D2
:103A0300679569FFE5669568FE22C3E49569CF74FF
:103A1300049568CF2567CF3566FE2231FEC374FF58
:103A23009FFF74039EFE228B4B8A4C894D8C4E8DD7
:103A33004FC3E54E94024006754E02754F00511E6A
:103A4300E54F2405FDE4354EFCC3EF9DEE9C50137A
:103A53000569E56970020568FFE5685403F5688F39
:103A63006980DBC3E49567F55174049566F550C32B
:103A7300E551954FE550954E4008AE4EAF4F51D7A7
:103A83008026AE50AF5151D7120126C3E54F955151
:103A9300FFE54E9550FEAB4BE54D2551F9E54C3511
:103AA30050FA78017C007D01120126E567254FFF5E
:103AB300E566354E5403F5668F6731FE8E4E8F4FA4
:103AC300D3E54F9401E54E94034008D20E900000D5
:103AD300740AF02274012567F974003566A801FCA5
:103AE3007D01AB4BAA4CA94D228B4B8A4C894D8D42
:103AF3004EC3E49569F55074049568F54FAF4E7E57
:103B030000C3E5509FE54F9E4015E5679569FDE5C8
:103B1300669568FCC3ED9FEC9E4004718C802E710A
:103B23009F502F716FC3E5679FE5669E4024AE4F9C
:103B3300AF50718C120126716FE54D2550F9E54C9C
:103B4300354FA801FCAD4B7B017A007901120126A8
:103B5300800BAF4E7E007D0051E50206967E00E5A8
:103B630069254EFFEE717A5002C20E22C3E54E95CF
:103B730050FFE4954FFE2235685403F5688F693191
:103B8300FEC3EF9401EE94032274012569F97400D6
:103B93003568FA7B01A84DAC4CAD4B22C3E5679564
:103BA30069E5669568227DFF1226F07B007A00792D
:103BB300000222907D007C00916B1204B23C4B000A
:103BC3000009603C46000012C03C3E000025803CDA
:103BD30039000038403C3400004B003C27000070A3
:103BE300803C22000096003C1D0000E1003C1000D8
:103BF30001C2003C0B000384003C060007080000E0
:103C0300003C58758DCC8008758D988003758D3078
:103C1300E58E54F44408F58E804C758D98800875B4
:103C23008D648003758D30E58E54F44401F58E80E8
:103C330035758D988008758D758003758D30538E1D
:103C4300F48023758D988003758D30E58E54F4448C
:103C530002F58E8011758D30538EF4E475318075C5
:103C63003025F52FF52E21E48F318E308D2F8C2EBC
:103C7300228F447B007A0079447D017C00412AC273
:103C83008EC2AB759810D29C7F807E2571B7538E00
:103C9300F0758BFF53890F438920900797E0440108
:103CA300F054FDF054FBF0E4900791F0A3F0A3F07F
:103CB300A3F0A3F0A3F0C299C298D2ACD2BCD2991C
:103CC300D28E22EF24F7604024F7603624ED603E65
:103CD30024ED602824ED601E24DB601424DA600ADE
:103CE30024B5702A7F007EE180287F007E968022A3
:103CF3007F807E70801C7F007E4B80167F407E38E5
:103D030080107FC07E12800A7F607E0980047F80DE
:103D13007E2571B7EEFF22C0E0C0F0C083C082C031
:103D2300D075D000C00730982FC298900795E0C394
:103D330094CF40089005F0E599F0805C900792E0FD
:103D430024F1F582E43405F583E599F0900792B107
:103D5300A8F0900795E004F030993DC29990079739
:103D6300E0FFC31330E003EF802B900796E0D3947A
:103D730000401E900793E024C1F582E43406F583E6
:103D8300E0F599900793B1A8F0900796E014F080BE
:103D930007900797E04401F0D007D0D0D082D083BA
:103DA300D0F0D0E032E004F0E075F0D084E5F0220A
:103DB300D19AFA7B018B24F52589269001A412015F
:103DC3006570037FFF22C2ACAB24AA25A92690010C
:103DD300A0120165F582758300120165FF9001A0B1
:103DE3007401120192E924A0D10FB1AC1201C5AB49
:103DF30024AA25A9269001A474FF120192D2AC43F0
:103E0300E70253D23F53E5FD22E924A6F9EA340140
:103E1300FA02014C8B278A2889298C2A8D2B7888D2
:103E230076010876050876F1121FF5C3E52B94CECB
:103E3300E52A94004004E4FEFF22C2ACD184F99049
:103E430001A5E41201D7AE2AAF2BD18424D0F9E423
:103E53003AA801FCAD03AB27AA28A929120126D150
:103E630084F99001A2E41201D7AF2B9001A3EF12C2
:103E730001D79001A51201D7D10CD192AE2AAF2B55
:103E8300227888860308E6FA08E622E4FFA1B35401
:103E9300FD1201C5D2AC227E007C017DA71201F97F
:103EA30074F12FF974053E22E4FFD1E26011E5239A
:103EB300600D5418FFBF0807D1EBE4FF1227327FD0
:103EC30001D1E26011E523600D5418FFBF0807D14B
:103ED300EB7F01122732D1F55004D18E80F82212E4
:103EE3001FDE8F23E523F4227B017A077998752F50
:103EF3007F22900795E0D394004003D38001C3222F
:103F0300C0E0C0F0C083C082C0D075D000C000C084
:103F130001C002C003C004C005C006C007E5962067
:103F2300E7FB759686E59620E7FB85975CE596208B
:103F3300E7FB759682E59620E7FB85975DE596207E
:103F4300E7FB759684E59620E7FB85975EE55C3095
:103F5300E102F197E55C30E202F1A9E55D30E003AF
:103F630012143AE55D30E102F1C4E55E30E203127A
:103F73004066E55C30E002F1A0D007D006D005D062
:103F830004D003D002D001D000D0D0D082D083D0CF
:103F9300F0D0E0320560E5607002055F220560E560
:103FA300607002055F2290089B7402F0E59620E79B
:103FB300FB759601759701E4F56A756B03756C03E0
:103FC30022E59620E7FB75960E759701E59620E7A7
:103FD300FB759691E59620E7FBAF97E56BB4030C71
:103FE300E59620E7FB75961175971022EF30E50BE8
:103FF300E59620E7FB759611759740EF30E20BE5E8
:104003009620E7FB759611E4F5977B017A05793BDA
:104013007D407C007F211127E59620E7FB759611F3
:10402300759701228C618D628B638A648965E56271
:104033004561602EE59620E7FB8F96E4FFFEC3EF14
:104043009562EE9561501BAB63AA64A9658F828E5E
:1040530083120165F597E59620E7FB0FBF00010E7C
:1040630080DC22E4FFE59620E7FB75960E75970248
:10407300E59620E7FB759694E59620E7FBAE97E57A
:104083006CB4030CE59620E7FB7596147597202214
:10409300EE30E60BE59620E7FB759614759780E501
:1040A3009620E7FB759696E59620E7FBAF97EF64BE
:1040B30040600DE59620E7FB759616759710800E08
:1040C3007B017A05797B7D407C007F2211DDE596BB
:1040D30020E7FB759614E4F597228C618D628B6360
:1040E3008A648965E5624561604B8F964396C0E4B7
:1040F300FFFEE56224FFFDE56134FFFCC3EF9DEEA7
:104103009C501BE59620E7FBAB63AA64A9658F82ED
:104113008E83E5971201D70FBF00010E80D4E4F51B
:1041230096E59620E7FBAB63AA64A9658F828E832D
:10413300E5971201D72253903B43A03DD29553A15B
:10414300CF75A27FC2A512199AD2A52275D6FF7583
:10415300D5FF75D48C75F3FD75F2FF75F1FF43A49C
:10416300C153A4F375A5C775A6FD75E103E4F5E294
:1041730043E2402275A2F075A140E4F5F8D2F9D2EA
:10418300F8C2FF2243B203E4F5B943B980122FB357
:1041930043B9C0122FB3E5B930E5FB75A90343B6A4
:1041A3009022E59620E7FB759601759708E5962022
:1041B300E7FB759607759707E59620E7FB75960964
:1041C300759707E59620E7FB75960B75970775D7E7
:1041D300E0E59620E7FB75960F75978043E602D2DC
:1041E300AFE59620E7FB75960175970122D2A7E408
:1041F300F53DF53E122FB3053EE53E7002053DC386
:104203009458E53D6480948240EAC2A7E4F53DF505
:104213003E122FB3053EE53E7002053DC394B0E563
:104223003D6480948440EAD2A722C2A832788412E3
:10423300044600000000E4F5C8538E0F75CBF075FB
:10424300CA5C74FFF5CDF5CCD2ADD2CA22C0E0C0B2
:10425300F0C083C082C0D075D000C000C001C002CE
:10426300C004C005C006C00778841203F5E4FAF958
:10427300F8EF2401FFEA3EFEE93DFDE83CFC7884CB
:1042830012042EC2CFD007D006D005D004D002D05E
:1042930001D000D0D0D082D083D0F0D0E032E47807
:1042A30082F608F675D10775BB1E75BA1F75BCFC7F
:1042B30075E8C243E60822C0E0C0D075D000C00054
:1042C300C001C005C006C007E5BBB41E1BAFBEEFEF
:1042D300FEADBDED7806CEC313CE13D8F97981F7C1
:1042E300EE19F775BB098019AFBEEFFEADBDED78D2
:1042F30006CEC313CE13D8F97983F7EE19F775BB3E
:104303001EC2EDD007D006D005D001D000D0D0D04A
:10431300E0328E3D8F3EE53E7803CEC313CE13D8F5
:10432300F97A00793F1236FA754BFF754C0C754DCF
:10433300DB853D4E853E4F7B017A05790E12078B57
:104343007B017A05790EE53F121FD37F018F408BE6
:10435300418A428943E540B4010790057BE020E0B0
:104363005090051974AAF0A3F071B5754C02AF40D3
:10437300122506AB41AA42A9431200038F4CAB415D
:10438300AA42A943AF40122506754BFF754C0C7525
:104393004DE485475185465085454F85444E71B55B
:1043A30012078B71B51200038F4C71B5AF40122504
:1043B30006227B017A05791922122ED67F007E0010
:1043C3007D057C000227F28B318A328933E4F53490
:1043D300FFFE1234FA8F828E83120165FDE4FBFA2D
:1043E300E534C313F534ED30E003433480EDC313F8
:1043F300FDE53430E10363349A0BBB00010AEB643F
:10440300084A70DC0FBF00010EEF64044E70C3AFA7
:10441300342212014C54C0FFBFC00971CAEF7004AB
:10442300FE7F0122E4FEFF228E288F2953281FE5F9
:1044330029AE287803CEC313CE13D8F97A00792A8C
:104443001236FAE5291237DE8002C333D8FCFF5552
:104453002A6F7F0160027F0022E4121FD7F5437A9F
:1044630005793B75470175480575493B754A407F9A
:1044730002122EEE900543E0B4FF127B017A057918
:104483003B754500754640E4FFFE1237099005432E
:10449300E0B4FF02E4F0900543E05402F0E044404E
:1044A300F090053DE054FEF0E4900549F090055589
:1044B300F0A3F0900558F0900544F02290053DE0FC
:1044C30054FBF0787DE654FEF6E49005EFF0227A93
:1044D30005795975470175480575495990058CE06B
:1044E300F54A227F407D007B011206967E002278EA
:1044F3006B7C057D017B017E0012012690053DE06A
:10450300227BFF7A0C79D9122290051BE51BD394E9
:104513002822541FF528E4F527F526AE28AF297B7A
:10452300012293FB740193FA740293228523478536
:104533002448852549900585E0F54A221201C5AB3B
:1045430029AA2AA92B22E0FEA3E0FFE48F478E4687
:10455300F545F5442290057DE0900549F022E525D7
:1045630025E024A2F582E43408F5832275F003A440
:10457300C58325F0C58322F528E5275407F527E4ED
:1045830022E52DFFE52C540FFEE42274FEF07BFFA1
:104593007A0C79B722900543E054CF22E07550009E
:1045A300F551A3E02290050AE0FEA3E0FF221228C2
:1045B300447F5002199A54DFF0E04410F0221204B1
:1045C3003A900543E022E0F54EA3E0F54F227BFF4E
:1045D300122290C20A229005BBE0D3940022120457
:0D45E30001D30203D1AF17121FDE8F182283
:10F800008F088D098B0A75E70075E60075A800530F
:10F81000B2FCD291D290C20D007F03318000539090
:10F820003B43A03DD295750F00751000C3E50F94C2
:10F83000F8504AAE0FAF108E118F1275B7A575B77D
:10F84000F1438F03AE11AF128F828E83E4F0538F9A
:10F85000FC750C00E50CC394FF5013750D00E50D0D
:10F86000C394FF500500050D80F4050C80E6B290AE
:10F87000E42510F5107402350FF50F80AF7F0131CC
:10F8800080750B00E50BC394FF5021750C00E50C4F
:10F89000C394FF5013750D00E50DC394FF50050090
:10F8A000050D80F4050C80E6050B80D853903B4392
:10F8B000A03DD2954390C07F033173AF083173AF41
:10F8C000093173AF0A3173C291750F00751000C30F
:10F8D000E50F94F840022157E51064007004E50F2D
:10F8E00064406016E51064007004E50F6480600AEF
:10F8F000E510B40007E50FB4C002B2917F00317388
:10F900008F0EE510450F700AE50E64026004D20DFB
:10F910008045AE0FAF108E118F12AE0FAF108E1349
:10F920008F1475B7A575B7F1438F01AE11AF128F64
:10F93000828E83E50EF0538FFEAE13AF148F828E4E
:10F9400083E493FFE50E6F6004D20D800A0510E595
:10F95000107002050F01CF53903B43A03DD295306C
:10F960000D047F0280027F00318000C291C290436B
:10F97000EF90228F1FC2FF851FA330FFFDAFA32290
:10F980008F6E53903B43A03DD295C2A5AF6E3173AD
:09F9900053903B43A03DD29522A7
:00000001FF
